:0300000002116387
:0C11630078FFE4F6D8FD7581EA0211AABD
:0100320022AB
:061A17008B288A29892AB0
:101A1D00751A027F48121BBB121D93EF20E0F9AB24
:101A2D0028AA29A92A1207207898E6FE08E6FDEDD6
:011A3D00FFA9
:011A3E002285
:100F3100434647002D53322D0052415445434C52F4
:100F410020554E49544C49544554524947545245F1
:100F5100565354525453544F505A45524F4241558F
:100F61004444464C54534156455253542050432017
:100F7100205F3120735F3220735F3520733120731E
:100F810020322073203520732031302073333020FC
:100F91007331206D2032206D2035206D20313020BD
:100FA1006D3330206D312068200000000100020007
:100FB10005000A001400320064012C025804B00B31
:100FC100B8177046508CA0010204081030466565C0
:100FD10074596172644D6574724F6666204F6E205C
:100FE100204E6F2020596573204F66662054696D2D
:100FF10065416C7420547269674F6666205472694A
:0910010067537472745265632098
:101AFD0025E024AAF582E4340FF58322052AE52A90
:101B0D00C3940222A62AE52A75F004A42208F60839
:041B1D00F608F622AE
:1013E700787276AB0876CD08760008760AE408F6B8
:1013F70008760108F6087664087640121B1A08F684
:101407007880F608760A08F608763C08F608761417
:1014170008F608760F121B1A788D760508F60876F7
:101427000A08F60876C808F608760C0876020876E1
:0A14370014087628087632021AD94C
:10196700751E1D751FC012166E7873E664CD700460
:1019770018E664AB60031213E7788CE6FFF46003A4
:0F198700EF7004788C7601788DE6B4FF02760558
:01199600222E
:0D1D4100C2AF7DC07C1DE4FF121C78D2AF44
:011D4E002272
:10166E007535FF851E36851F37753800753900753F
:10167E003A72E4FFAB35AA36A9378F827583001212
:10168E0006F3AB38AA39A93A8F8275830012073256
:10169E000FBF26E0788BE6FFF46003EF7004788BC3
:0216AE007601C3
:0116B0002217
:101AD9007D01E4FF121B62121D41C2AF7F727B269A
:101AE9007DC07C1D121C82D2AF7F0212182FE4FD2B
:041AF900FF021B626B
:10048000E4F5287BFF7A0F79311217767F05121871
:100490002FA297829650FAA2969218A2979219E5E7
:1004A0002875F004A4243AF9740F35F0FA7BFF1292
:1004B00017767F0512182F852829E4F52A7BFF7A05
:1004C0000F7935121776E528B40A00400302054E6D
:1004D0009004D7F82828730204F502054E02051689
:1004E00002051E02052202052A0205320205360215
:1004F000053E0205467F01EF121AFD7874E6FC08FE
:10050000E6FD7401936D7003E4936C70028F2A0F03
:10051000BF0FE40205D47876E6F52A0205F778776E
:100520008002787FE6F52A020611787EE6F52A0237
:10053000063F788880027889E6F52A02065C788A88
:10054000E6F52A020691788DE6F52A0206B7E52837
:100550006529600302049FA218309601B35013A2CC
:1005600096921830960C0528E528C3940D4003E4B4
:10057000F528A219309701B350D4A2979219309759
:10058000CDE528B40D0050C690058FF828287302D9
:1005900005B60205DF0205E502060302061D020696
:1005A0003102064A02066702067F0206A50206C855
:1005B0000206CE0206D4052AE52AC3940F4003752D
:1005C0002A01E52A121AFDE493FF7401937874CF8F
:1005D000F608EFF6121B13246EF9740F02069A1236
:1005E000149A02054E052AE52AC394034003E4F554
:1005F0002A7876A62AE52A75F004A424CEF9740F89
:1006000002069A121B094003E4F52A7877A62AE528
:100610002A75F004A424DAF9740F02069A121B0951
:100620004003E4F52A787F121B1124DAF9740F8055
:1006300069121B094003E4F52A787EA62AE52A758B
:10064000F004A424E2F9740F8050052AE52AC3942B
:10065000044003E4F52A7888A62AE52A75F004A464
:1006600024EAF9740F8033052AE52AC39403400372
:10067000E4F52A7889121B1124EAF9740F801B050E
:100680002AE52AC394044003E4F52A788AA62AE5D9
:100690002A75F004A424FAF9740F35F0FA7BFF12DE
:1006A000177602054E052AE52AC394064003E4F5B1
:1006B0002A788DA62AE52A900FC89375F018A4FF12
:1006C000AEF012136F02054E1213E702054E121A16
:0A06D000D902054E43A20802054EB0
:0A1D76004552415300444F4E450012
:101D12007874E6F54D08E6F54E22E561AE60780688
:011D2200229E
:1011EF00C216C217788CE6FFE4FCFDFEFB7A20F9ED
:1011FF00F81207668F678E668D658C64E47B40FA04
:10120F00F9F81207F18E5E8F5FE4F529F52AC3E531
:10121F002A955FE529955E501CE52864816016AF1D
:10122F002AAE29121997121C648F28052AE52A70F5
:10123F00DD052980D9E528B48108E52A152A700231
:10124F001529E52A655F7004E529655E700CD216D5
:10125F00121D4FE4F560F5618007852960852A61CD
:0B126F00E4F562F563754C80121D125F
:01127A002251
:10199700C3EF955FEE955E5024EF7806C333CE33E1
:1019A700CED8F9FD751A02EE7898F6CFEDCFEF088D
:0D19B700F67F50121C0B121D93EF20E0F97B
:0119C4002200
:031BF100CDEFCD68
:101BF400751A02EE7898F6ED08F67F50121C0B1257
:061C04001D93EF20E0F942
:011C0A0022B7
:101C6400751A017F50121BBB121D93EF20E0F97807
:031C740098E6FFF0
:011C7700224A
:101C4F00121BF1E4FFFE0FBF00010EBE0FF8BFA085
:041C5F00F5121C64FA
:011C6300225E
:06186500CBEFCBCAEECA76
:10186B00301603301727751A03EA7898F6EB08F64B
:10187B0008EDF67F50121C0B121D93EF20E0F9E4DC
:0D188B00FFFE0FBF00010EBE0FF8BFA0F55D
:01189800222D
:1016F400752B00752C00752D4CE4F52A121D1CC3A6
:1017040033CE33CED8F97C00252AFFEC3EFEAB2B3A
:10171400AA2CA92D852A827583001206F3FD1218BE
:1017240065052AE52AC3940640D2756200756306EE
:011734002292
:1012F7008E288F29121D1CC333CE33CED8F9256310
:10130700FFE5623EFEEEC0E0EFC0E0E528FDD0E07D
:10131700FFD0E0FE1218650563E5637002056212EF
:101327001D1CC333CE33CED8F92563FFE5623EFEDD
:10133700AD291218650563E563700205620550E57E
:10134700507002054FC3E5639440E562940040176F
:10135700E4F562F5630561E56170020560955FE597
:0813670060955E4002D21622DF
:10149A00E4F562F5637BFF7A1D7976121776D21727
:1014AA00E4F535F536C3E536955FE535955E5021A9
:1014BA00E536AE357806C333CE33CED8F9F5638E2A
:1014CA00627D81FF1218650536E53670D8053580CC
:1014DA00D4C2177BFF7A1D797B121776E4F560F583
:0714EA0061F562F563C21613
:0114F10022D8
:10144100E4F535F536F537F538C3E538955FE53719
:10145100955E5044E5366481603EAF38AE3712196F
:1014610097121C648F36E53664807022AF350535DE
:10147100FCFDFEFBFAF9120D087F2C121D99AE3707
:10148100AF38E4FCFDFBFAF9120D08121D8A05388C
:08149100E53870B5053780B1A4
:011499002230
:0215E3008F3542
:1015E500E4F536F537F538F539C3E539955FE5386E
:1015F500955E5030E5376481602AAF39AE381219EF
:1016050097121C648F37E537B4800FE53665357062
:1016150007AF39AE3802199705360539E53970C96E
:04162500053880C53F
:01162900229E
:10173500121D12787FE6F551E4F54FF5501216F4B7
:101745008560688561697F01121A8D30021A788279
:10175500E6FE08E6FFE4FCFD7B64FAF9F81207668D
:101765008F5D8E5C8D5B8C5A300505C205121C3968
:011775002251
:1017F500856028856129E563456260080529E52935
:10180500700205288568608569611216F48528606F
:10181500852961C3E529955FE528955E4007E4F5CF
:0A18250060F561D2167F02021A8DF1
:101C7800740478FF769612FF0322740078FF769634
:041C880012FF032222
:0300330002100AAE
:0D100A00C0E0C0F0C083C082C0D075D00827
:10101700E5D954F8FF12090A104408104410105378
:1010270018106E20105528106E301070381076404A
:10103700106E48108F5010AC58000010BA851DDA9A
:10104700C2DDC2DC751B00751C008070800EE51ABE
:1010570070028056051CE51C7002051B12000E8FDE
:10106700DAC2DDC2DC80558016D2DDC2DC804DC21B
:10107700DDC2DCE51A7004C2DA8041D2DA803DC2F3
:10108700DDD2DC7518048034AFDA120026051CE5C2
:101097001C7002051BC2DDC2DCE51A7004C2DA80CF
:1010A7001BD2DA8017AFDA120026C2DDD2DC751840
:0E10B700028009751804C2DDC2DCD2DAC2DB89
:0B10C500D0D0D082D083D0F0D0E03239
:1019C50043910C43920CE4F5DBEF25E0F5DB301891
:1019D5000343DB0175DD1775DC1775D84453F8FE35
:0919E50053F7FEE4F518D2E822E4
:101C0B00E51830E002FF22E4F519751803EF25E023
:071C1B00F51DD2DD7F02225E
:101BBB00E51830E002FF22E4F519151A751805EF48
:0B1BCB0025E04401F51DD2DD7F022261
:061D930020DBFDAF182269
:0D000E00151AAF19051974982FF8E6FF2296
:0C00260074982519F8EFF60519151A2238
:101CEE00E4F5847585FF53912F759210F5A475A5B3
:021CFE00FF22C3
:101A66006F035D5733767E437F771004007B3E6CB1
:101A76001F7C78773B020F382C5A1A6F79751876C7
:071A86003C0E2F4E2B375DD3
:101901004EFECCEFCC0F74982CF8EEF6EDC43322DA
:10191100901A72E493FF78E2F608EFF608F608F6FB
:1019210022E493FF74E22EF8EFF60E22EE3395E0F7
:03193100FDFC2298
:1010D000E4FF0F2498F876CD0F74982401F87680F9
:1010E0000F74982402F876E00F74982403F876F8C9
:1010F000301A0A0F74982404F87671800ACEEFCE65
:101100000F74982EF8767078E2E6FEC4540FFDCC8A
:10111000EFCC0F74982CF8EDF6EEC454F0FE78E3A3
:10112000E6FD131313541F12190154E0FE78E4E690
:10113000FD1313543F1219013354C0FE78E5E6FD48
:10114000C31312190133335480FECDEFCD0F7498C1
:101150002DF8EEF68F1A7F38121C0B121D93EF201C
:02116000E0F9B4
:01116200226A
:10189900C21A121911751A0A789876CD0876800835
:1018A90076E00876F80876700876050876D5087621
:1018B9009B0876FFE408F67F38121C0B121D93EF84
:0318C90020E0F923
:0118CC0022F9
:101BD600EF24F9600B14600C2402700EC21A800701
:0B1BE600D21A80031219111210D02235
:1014F200C3EF648094E1400ED3EF648094FA500607
:10150200EF24ACFF803CC3EF648094C1400ED3EF64
:10151200648094DA5006EF24CCFF8026C3EF648007
:1015220094B0400ED3EF648094B9500674D02FFF6C
:101532008010BF2D047F0A8009BF5F047F0B8002E9
:031542007F0C22F9
:101A3F00CEEDCECDEFCDCFEECF1214F2EF3395E04A
:101A4F00FE74662FF582741A3EF583E493FF74E2F9
:071A5F002DF8EFF60210D094
:061776008B378A38893927
:10177C00E4FE901A72121922BE04F7E4FEAB37AAEB
:10178C0038A9398E827583001206F3FF6019121482
:10179C00F2EFFD3395E0FC74662DF582741A3CF57E
:0A17AC0083121922BE04D60210D0E9
:04136F008F828E8358
:1013730012192D7B197AFC79FF78FFD3120891405B
:101383000390FC19AF82AE8312192DE47B0F7A27E9
:10139300F9F8C3120891500390270FE4F52B74DD7D
:1013A300252BF8E4F6052BE52BB405F2AE83AF82CB
:1013B30012192D7B007A0079DD120D0878E0E670B2
:1013C3001A752B0374DC252BF8E6FF74DD252BF847
:1013D300EFF6D52BEF78DD762080E17B007A00797C
:0413E300DD0217769A
:101CC800C213C215C212E4FDFF121B62E4FD7F01BC
:031CD800021B628A
:101B6200EF146011047016BD0104C2A78002D2A74F
:0E1B7200A2A7921422BD0103C2A622D2A6226F
:101A8D00EF24FE600D14601124027019D213756BD2
:101A9D000122C213A21492A722D215756C027D01E8
:061AAD007F01121B622202
:1019EE00301312D56B0F30A707C2A7756B0F80058A
:1019FE00D2A7756B23E56CD39400400CD56C09C24D
:091A0E0015E4FD7F01121B6222A8
:0F1D320046554C4C005A4C4F470020332D330080
:071D6B00C191015201C10EFC
:101B2100E6FE08E6FFE4FCFD22E5549618E6648033
:101B3100F8E5536480982278D31208CC78CB020858
:011B4100E5BE
:02182F008F36F2
:10183100E4F537F538C3E5389536E537940050239C
:10184100900000AF82AE83E4FCFD7B207A4EF9F874
:10185100D31208914003A380EA0538E53870D60514
:031861003780D2FB
:011864002261
:0E1D4F007BFF7A1D79321217767F0A02182F59
:0F1D2300D20B301606121D4FC20B22121735229B
:05001E00C20B0217F502
:101C390078D71208F100000000121B3878D3120877
:061C4900F1000000002282
:10003600121CEE121D80121CC87F0412182F209766
:100046000B7D017F0112127BD2AF80FE209612D269
:10005600AF121967C2187F701219C51211EF120478
:1000660080121967788DE6FDE4FF12127BD2AFC2CB
:10007600187F701219C57F0112182F1211EF12186E
:10008600997A1D79371204757A1D793C1204751216
:100096000032E4F56D1219347F0112182FE478DB73
:1000A600F608F6121D9CA2969208A2979209E4F50C
:1000B6002478CF1208F100000000E4F52578D71265
:1000C60008F1FFFFD8F178CB1208F100000000E438
:1000D600F54A78D31208F100000000C20CC20BE406
:1000E600F526F5277895E6F54BE4F555C20F788E9B
:1000F600E6F55308E6F554E4F559F558F557F5567F
:10010600F55DF55CF55BF55AF5207877E66004D287
:10011600808002C2807888E624FE600B14600C247E
:1001260002700AD2018006D2068002D2007889E6E1
:1001360024FE6007047006D2028002D207788AE69F
:1001460024FE600B14600C2402700AD2038006D2CF
:10015600048002D205300117C2017880121B217B70
:1001660064FAF9F81207668F598E588D578C56E542
:100176006DC3940240F9E4F56D209605209702D2EE
:100186001030963530973230102FC21078CB1208C7
:10019600CCEC4D4E4F78D7700C1208F100000000E1
:1001A600121B3880101208F10000000078CB1208EC
:1001B600F100000000D209D208A208309601B3501F
:1001C6001FA2969208309618201015C201E54A60C3
:1001D60007E4F54A7F068005754A017F07121BD69C
:1001E600A209309701B35017A297920930971020B1
:1001F600100DB20B300B05121D23800312001E12C8
:100206000930AF59AE58AD57AC56EC4D4E4F60263F
:1002160074FF2FF559EE34FFF558ED34FFF557EC22
:1002260034FFF556AF59AE58AD57FC4D4E4F7006DC
:10023600200B03121D23AF5DAE5CAD5BAC5AEC4DDB
:100246004E4F602374FF2FF55DEE34FFF55CED3401
:10025600FFF55BEC34FFF55AAF5DAE5CAD5BFC4D74
:100266004E4F700312001EE5556008D5550578956A
:10027600E6F54B0525E525C39401500302046FE41A
:10028600F525FB7A0079E6121A1778E7EEF608EFFD
:10029600F678E6E66402600302046F78CF1208D8A7
:1002A600E8C0E0E9C0E0EAC0E0EBC0E078E7E6FEDF
:1002B60008E6FF7876E6FD121597D0E0FBD0E0FA67
:1002C600D0E0F9D0E0F8EB2FFFEA3EFEE93DFDE88D
:1002D6003CFC78CF1208E50524E524C394055003B9
:1002E60002046F78CF1208CCE47B05FAF9F81216EF
:1002F6002A78CF1208E578CF1208CC78CB1208D826
:10030600C3EF9BFFEE9AFEED99FDEC98FC78CF12B9
:1003160008E578D71208CC78CF1208D8D3120891FE
:10032600400A78CF1208CC78D71208E5E54A600D66
:1003360078D9E6FF08E678E9CFF608EFF678D1E651
:10034600FF08E678E7CFF608EFF6301150C3E695DA
:1003560054FF18E69553FE121D007894E6FDD3EF80
:100366009D7480F86E985035D20FD20DC3789112D5
:100376001B2A40037552FFD3788F121B2A50037530
:100386005201AF52EF3395E0FE7892E6FC08E6FDA7
:10039600120754EF2554F554EE3553F553300F0E2E
:1003A6007F03121A8D7896E6F54B08E6F555E54A71
:1003B600600478E9800278E7E6FE08E6FF12136F2C
:1003C6000527E52770020526C3787596E526189653
:1003D6004045E4F526F527300C0F78E7E608FF12CE
:1003E6001D9978E8E6FF121D99300B2B7F03121A30
:1003F6008D20161D787FE6600C300D09C20D7F003A
:100406007E821212F778E7E6FE08E6FF1212F78000
:1004160006121D4F12001E78CF1208CC78D3120890
:10042600E578CF1208F100000000E4F524C20F3091
:100436000405C204121C393006167884121B217872
:10044600D31208D8D31208914006200B03121D239D
:100456003007167886121B2178D31208D8C31208E3
:0F046600915006300B0312001E1219EE020175A1
:0B0475007BFF1217767F0412182F2265
:101AB300444C0021536967005A4C4F47004D4F4433
:101AC30000332D3300466562203134203230303606
:061AD3000050524F4700D5
:1016B100AF30AE2FAD2EAC2DEC4D4E4F22EF24FFAF
:1016C100F530EE34FFF52FED34FFF52EEC34FFF558
:1016D1002D22E4753020752F4EF52EF52D22E4755F
:1016E1003001F52FF52EF52D22752A00752B007589
:0316F1002C722236
:10093000121D5DEF7003020B3C121B9EE4F54AEFA3
:1009400012090A0B1C240B252A0B28500A7A52097B
:100950006E6109FC630B3A640A4F6C0A55720A52C5
:10096000730A7E740AEC760AE97800000B3C7BFF80
:100970007A1A79B31217761216D3121D5DEF700A28
:100980001216B160051216BE80F01216B170030285
:100990000B3C121B9E8F291215E3E4F5301216E36F
:1009A000E47F06FEFDFCAB30AA2FA92EA82DC312B2
:1009B00008A7501F121C648F29121D99E5302401CD
:1009C000F530E4352FF52FE4352EF52EE4352DF5F1
:1009D0002D80CD121C648F29E52964806016E529DD
:1009E00064816010121D99121C648F29121D997563
:1009F00028018003E4F528E52870D8221216EA12AF
:100A000016DFF5291216B160241216D3121D5DEF00
:100A1000700A1216B160051216BE80F01216B1608F
:100A200003120B3D0529E529C3942640D71216B1C0
:100A3000601A7872B6AB0708B6CD03020B227BFFB3
:100A40007A1A79B61217767F0A02182F020AE6B2CE
:100A50000C220214411216EAE4F529AB2A052CE512
:100A60002CAA2B7002052B14F91206DAFF121D991D
:100A70000529E529C3942640E22243A20822752ACB
:100A800000752B00752C701216DFF5291216B16057
:100A9000241216D3121D5DEF700A1216B1600512F2
:100AA00016BE80F01216B16003120B3D0529E52930
:100AB000C3940240D71216B1602CAE70AF71EE3302
:100AC00095E0FDFC78D31208D8C3EF9BF534EE9A7D
:100AD000F533ED99F532EC98F531AF34787CE533A8
:100AE000F608EFF6803C02166E02149A7A1A79BB69
:100AF000120B517A1A79C0121CDB788BE62430FF76
:100B0000121D99121D8A7F76121D997A1A79C412C4
:100B10000B517A1A79C8121CDB021D8AE4787CF624
:100B200008F6021AD90213E77BFF7A1A79D4121752
:0C0B3000767D017F0112127B80FED20E48
:100B3C0022121B9EAB2AAA2BA92C85298275830015
:100B4C00EF120732227BFF121CDB121D8A7BFF2265
:0A1D8000E4F5955396BF53A27F22AD
:031D7200016E00FF
:101934005389F0438901538FFE758C70E4F58A5303
:10194400B8FD53B7FDD2A9D28C53890F43891053E4
:101954008FEF758DFF758B4753B8F753B7F7D2AB3D
:03196400D28E22FE
:03000B00021C22B2
:101C2200C0E0056D758C70758A00056FE56F30E058
:071C320003854B6ED0E03288
:03001B00021B8045
:101B8000C0E0C0D0758DFF758B47E56ED3940040E3
:0E1B900006D294156E8002C294D0D0D0E032FE
:101C8C000D0A00303132333435363738394142435E
:041C9C004445460075
:101CA000AF49AB3DAA3EA93F054922AF3CAE3BAD93
:041CB0003AAC3922EF
:10127B005387BF75985053877FE4F5BABF01054379
:10128B00A240800353A2BFE4F5BDED1460151460BA
:10129B001A14601F1460242404702575BEF075BFEA
:1012AB000B802375BEF075BF05801B75BEF075BF37
:1012BB0002801375BE7075BF01800B75BEB08003C5
:1012CB0075BE30E4F5BF75BD035391FE43920143E8
:1012DB0091025392FDC21B53B8EF53B7EF43B810B3
:0C12EB00E478C9F618F678CAF6D2AC22F6
:030023000218CDF3
:1018CD00C0E0C0D075D01030981E78C9E6C3940F13
:1018DD00501418E60624B8F8A69978C90618E6C378
:1018ED00941040027600C298309904C299C21BD060
:0418FD00D0D0E03235
:08000300201BFDD21B8F992286
:101B420078C9E6D39400401508E60624B8F8E6FF03
:0F1B520078C91608E6C394104005E4F6227F0018
:011B61002261
:031D990002000342
:101B9E007F207E4E78C9E67010D3EF9400EE94004D
:0C1BAE004007EF1F70EE1E80EB121B4280
:011BBA002208
:101CDB001206DAFF600C121D99740129F9E43AFA25
:031CEB0080EE2266
:0E1D5D0078C9E6D3940040037F01227F002264
:091D8A007BFF7A1C798C021CDB42
:0E0D08008F3C8E3B8D3A8C398B3D8A3E893F65
:100D1600E4F549EC4D4E4F7017E94A4B70057F30AC
:100D2600021D99121CA08F827583007430020E2B4F
:100D3600121CADEC33502AE53F453E453D70077F1A
:100D46002D121D99800D121CA08F82758300742DA3
:100D5600120732121CAB1208838F3C8E3B8D3A8CE5
:100D6600397548017543007542CA75419A75403B0D
:100D7600E4FFFEFDFCAB43AA42A941A840D31208FA
:100D8600A75003020E16121CABA8401207F18F479C
:100D96008E468D458C44EC4D4E4F7004E5487023CD
:100DA600E5472430FFE53F453E453D7005121D9958
:100DB600800EAE49121CA28E82758300EF12073296
:100DC600E4F548AF43AE42AD41AC40AB47AA46A9B5
:100DD60045A844120766C8ECC8C9EDC9CAEECAC31D
:100DE600E53C9FF53CE53B9AF53BE53A99F53AE556
:100DF6003998F539AF43AE42AD41AC40E47B0AFACF
:100E0600F9F81207F18F438E428D418C40020D7620
:100E1600E53E453F453D6010AB3DAA3EA93F8549AD
:080E260082758300E41207321B
:010E2E0022A1
:100B5C000134C35001DBBF68028BBB800344B798E0
:100B6C000407B3B004D5AFC805A9ABE00689A7F854
:100B7C000775A410086DA02809719C400A8198582B
:100B8C000B9F94700CCA90880DE98CF90E048CA004
:100B9C000EA88AAC0F4D88B80FF786C410A184D06C
:100BAC00115182DC120580E812BB7EF413747D00B7
:100BBC0014307B0C14F2791815B877241680753024
:100BCC00174B733C1819714818ED6F5419C46D60AC
:100BDC001AA16B6C1B7E69781C6167841D4A659039
:100BEC001E37639C1F2561A8201A5FB421125DC0BB
:100BFC00220D5BCC230E59D8241557E4251F55F034
:100C0C00262F53FC27425208285B501429764E207D
:100C1C002A9B4C2C2BC04A382CEE48442E1E465096
:100C2C002F55445C308F426831D1407433173E806D
:100C3C0034633C8C35B13A98370938A4386636B0F1
:100C4C0039C734BC3B2D32C83C9D30D43E0F2EE00E
:100C5C003F882CEC41062AF8428D290444182710B1
:100C6C0045AB251C4741232848E121344A861F40C7
:100C7C004C311D4C4DE21B584F9C1964515D177043
:100C8C005323157C54EF138856C4119458A20FA00B
:100C9C005A830DAC5C6D0BB85E6009C4605807D00C
:100CAC00625A05DC646203E8667301F4688A00002A
:100CBC006AA1FE0C6CB8FC186ECFFA2470E6F83002
:100CCC000000000000000000000000000000000018
:100CDC000000000000000000000000000000000008
:100CEC0000000000000000000000000000000000F8
:0C0CFC00000000000000000000000000EC
:1017B60075F004E52FA4245CF582E5F0340BF5837F
:1017C600E49322FE740193FF75F004E52FA422F53D
:1017D60083C37401939FFFE4939EFEE4228F308EB1
:0F17E6002F8D2E8C2D228F2C8E2B8D2A8C29222D
:101CB400C3EF9DEE9C400AD3EF9BEE9A50037F0145
:041CC400227F002259
:040E2F008E2D8F2E47
:100E3300E4F52F1217B6FC740193FD1217CE24604C
:100E4300F582E5F0340BF583E493FA740193FBAF79
:100E53002EAE2D121CB4EF7003020F1F1217B61221
:100E630017C92460F582E5F0340B1217D58F338E42
:100E730032F531F5301217CE2462F582E5F0340BEA
:100E8300F583E4931217C9245EF582E5F0340B125F
:100E930017D58F378E36F535F534AD35AC341208AA
:100EA300838F378E368D358C34AE2DAF2EE4FCFD1B
:100EB300EEC0E0EFC0E01217B6FE740193FBCAEE7A
:100EC300CAD0E0FFD0E0FEC3EF9BFFEE9AFEED94A5
:100ED30000FDEC9400FCAB37AA36A935A834120701
:100EE30066AB33AA32A931A83012162AC8ECC8C996
:100EF300EDC9CAEECACBEFCB1217CE245EF582E55D
:100F0300F0340BF583E493FE740193FFE4FCFDEBF3
:100F13002FFFEA3EFEED39FDEC38FC22052FE52FCD
:0D0F2300C3946A5003020E36E4FFFEFDFC8D
:010F3000229E
:011D9C002224
:101545001217E3AB30AA2FA92EA82DE8C0E0787AB0
:10155500E6FE08E6FFE4FCFDD0E0F8120766121788
:10156500E3780E1208B81217E3787CE6FE08E6FF6A
:10157500EE3395E0FDFCE5302FF530E52F3EF52FF8
:10158500E52E3DF52EE52D3CF52DAF30AE2FAD2EDC
:02159500FC2236
:021597008D289D
:10159900120E2F1217EC1215451217ECE5281460DC
:1015A9001C14702DE47FE87E03FDFCAB2CAA2BA94B
:1015B9002AA829120766E47BE87A0B800CAF2CAEC7
:1015C9002BAD2AAC29E47B03FAF9F812162A121773
:0915D900ECAF2CAE2BAD2AAC29BD
:0115E20022E6
:10116F00020036E493A3F8E493A34003F68001F260
:10117F0008DFF48029E493A3F85407240CC8C33381
:10118F00C4540F4420C8834004F456800146F6DF50
:10119F00E4800B0102040810204080901D6BE47E58
:1011AF00019360BCA3FF543F30E509541FFEE49345
:1011BF00A360010ECF54C025E060A840B8E493A30C
:1011CF00FAE493A3F8E493A3C8C582C8CAC583CA37
:1011DF00F0A3C8C582C8CAC583CADFE9DEE780BEEF
:011D7500006D
:1006DA00BB010689828A83E0225002E722BBFE021E
:0906EA00E32289828A83E4932251
:1006F300BB010CE58229F582E5833AF583E02250BC
:1007030006E92582F8E622BBFE06E92582F8E22205
:0D071300E58229F582E5833AF583E493221F
:10072000BB010689828A83F0225002F722BBFE01B8
:02073000F322B2
:10073200F8BB010DE58229F582E5833AF583E8F0FD
:10074200225006E92582C8F622BBFE05E92582C8A9
:02075200F22291
:10075400EF8DF0A4A8F0CF8CF0A428CE8DF0A42EB9
:02076400FE2273
:10076600E88FF0A4CC8BF0A42CFCE98EF0A42CFC32
:100776008AF0EDA42CFCEA8EF0A4CDA8F08BF0A4B0
:100786002DCC3825F0FDE98FF0A42CCD35F0FCEB0F
:100796008EF0A4FEA9F0EB8FF0A4CFC5F02ECD39D4
:0F07A600FEE43CFCEAA42DCE35F0FDE43CFC2241
:1007B50075F008758200EF2FFFEE33FECD33CDCCFB
:1007C50033CCC58233C5829BED9AEC99E58298407E
:1007D5000CF582EE9BFEED9AFDEC99FC0FD5F0D65B
:1007E500E4CEFBE4CDFAE4CCF9A88222B800C1B985
:1007F5000059BA002DEC8BF084CFCECDFCE5F0CBC3
:10080500F97818EF2FFFEE33FEED33FDEC33FCEBFB
:1008150033FB10D703994004EB99FB0FD8E5E4F9B6
:10082500FA227818EF2FFFEE33FEED33FDEC33FCA3
:10083500C933C910D7059BE99A4007EC9BFCE99A97
:10084500F90FD8E0E4C9FAE4CCFB2275F010EF2FDC
:10085500FFEE33FEED33FDCC33CCC833C810D707DC
:100865009BEC9AE899400AED9BFDEC9AFCE899F817
:0E0875000FD5F0DAE4CDFBE4CCFAE4C8F922AA
:10162A00C2D5E830E70FB2D5E4C39BFBE49AFAE4EB
:10163A0099F9E498F8EC30E717B2D5121660120758
:10164A00F1E4C39BFBE49AFAE499F9E498F880037D
:10165A001207F130D50DE4C39FFFE49EFEE49DFD21
:04166A00E49CFC22DE
:0E088300C3E49FFFE49EFEE49DFDE49CFC2286
:10089100EB9FF5F0EA9E42F0E99D42F0EC6480C8DE
:0608A10064809845F0227E
:1008A700EB9FF5F0EA9E42F0E99D42F0E89C45F0A7
:0108B700221E
:1008B800E86010ECA2E713FCED13FDEE13FEEF1356
:0408C800FFD8F02243
:0C08CC00E6FC08E6FD08E6FE08E6FF2258
:0D08D800E6FB08E6F908E6FA08E6CBF82290
:0C08E500ECF608EDF608EEF608EFF6223F
:1008F100D083D082E493F608740193F608740293CE
:09090100F608740393F674047304
:10090A00D083D082F8E4937012740193700DA3A37C
:10091A0093F8740193F5828883E473740293686090
:06092A00EFA3A3A380DF90
:101D0000C3EE6480948040028007C3E49FFFE49E9A
:021D1000FE22B1
:00000001FF
